S0160000755461736B657256312E345F424D2E7372656358
S1132800FC05002051630000A95A00009F5A0000F3
S1132810A15A0000A35A0000A55A000000000000BD
S1132820000000000000000000000000AD5A00009D
S1132830A75A000000000000AB5A0000DD5B000056
S1132840AF5A0000AF5A0000AF5A0000AF5A000060
S1132850AF5A0000AF5A0000AF5A0000255D0000D7
S1132860AF5A0000AF5A0000AF5A0000AF5A000040
S1132870F55A0000AF5A0000AF5A0000AF5A0000EA
S1132880AF5A0000AF5A0000AF5A0000AF5A000020
S1132890F95B0000B15A0000AF5A0000AF5A0000C3
S11328A0AF5A0000AF5A0000AF5A0000AF5A000000
S11328B0DD5B0000AF5A0000AF5A0000C55C0000A9
S1132900084B202200B51A60074B084918700A7852
S113291052B2002AFBDA1878054B2022C0B21A60A2
S113292000BDC04608F00F40066007400060074045
S113293004F00F400B4B202210B51A600A4B18709C
S11329400A480278094C52B2002AFADA1878197047
S1132950C0B2227852B2002AFBDA1B78044B202240
S11329601A6010BD08F00F40066007400060074081
S113297004F00F400F4B30B520241C600E4B0F4D5C
S1132980187028780D4C40B20028FADA1878C0B2D2
S1132990013AD2B2FF2A08D00D781D7025786DB2A5
S11329A0002DFBDA1D780131F2E7054B20221A6075
S11329B030BDC04608F00F40066007400060074085
S11329C004F00F400F4B70B520241C600E4B0F4DCC
S11329D0187028780D4C40B20028FADA1878FF25D0
S11329E0C0B2013AD2B2FF2A08D01D70267876B25E
S11329F0002EFBDA1E780E700131F2E7044B202220
S1132A001A6070BD08F00F40066007400060074080
S1132A1004F00F4008B561202A2101F07FFF08BDB2
S1132A2008B56120292101F079FF08BD08B56120AE
S1132A307C2101F073FF08BD08B5054B10221A6014
S1132A400A212020FFF776FF892101F05EFF08BDEF
S1132A5048F00F4008B5144B188020280ED004D835
S1132A6000281CD008281DD119E0802817D0802305
S1132A705B00984208D0402814D110E061200B4933
S1132A80062202F067F90DE0962106226120C900B2
S1132A9002F060F9064B1A78064B1A7002E06120C6
S1132AA002F092F908BDC04630FEFF1F7017000007
S1132AB0F7FFFF1F0CFEFF1F08B5044B04491868FD
S1132AC04022183001F0BDFD002008BD1CFEFF1F90
S1132AD05C6B000000B5054B054A19781170FF22A4
S1132AE0002801D1034A12781A7000BD0CFEFF1FA2
S1132AF000FEFF1FF7FFFF1F024B1A78024B1A70EC
S1132B007047C04600FEFF1F0CFEFF1F30B51B4B75
S1132B1085B01B68011C0024684604725A1DD27FCC
S1132B20C272082282808022C280612202731A1C2F
S1132B304E32127842731A1C4F321278DB69827358
S1132B40201C6A46009301F055FC0D4D2870A042EC
S1132B5010D00521221C01F0ADFB009B5B0609D5BA
S1132B600849221C287801F0A5FB28788121221C21
S1132B7001F0A0FB287805B030BDC0461CFEFF1F45
S1132B80F7FFFF1F04040000F0B5CE4E807B3468CD
S1132B909DB00190002C00D0CBE0201C02F046FF39
S1132BA0582001F023FFC84B1860201CFFF784FF56
S1132BB080231B02984207D1962161200901032238
S1132BC002F0C8F8042300E00123336000F04EFD56
S1132BD06D20042102F088F80320FFF797FF0028F6
S1132BE000D1E4E1B94BBA481A78BA4B0CAC1A706C
S1132BF001F07AFEB84B0125122100270C93201C0A
S1132C008023A1712771A3606571E57103F020FC35
S1132C1009232371B14B201C0C93FF23E371202360
S1132C20A36003F015FCAE4B12220C930823A3609F
S1132C30AC4B2771A2716571E57119688022D203CA
S1132C400A431A60A84B50221A70A84B1D70A84B57
S1132C501B78A84B1B78FFF7EFFEFA20000102F067
S1132C6091FFA54BA54F1B685A0600D53D60A448AB
S1132C7001F03AFE06212620FFF75CFE0F212520F5
S1132C80FFF758FE9F4D0522291C2A20FFF772FEEC
S1132C909D4905222B20FFF76DFE9C4905222C201F
S1132CA0FFF768FE0522291C3020FFF763FE072189
S1132CB02220FFF73FFE07213C20FFF73BFE0721C0
S1132CC03D20FFF737FEE220FFF71AFEE120FFF771
S1132CD017FE27207021FFF72DFE3B688C4D002B3B
S1132CE012D08C4801F000FE18212420FFF722FEA8
S1132CF00A212020FFF71EFE10232B60612064218F
S1132D007B2202F027F808E0834801F0EDFD202043
S1132D100B21FFF70FFE10232B60201C03F098FB00
S1132D2007E0E5782279002D0CD1032A0DD103F0B8
S1132D30CFFA0CAC0198211C052201F0D1FA00282D
S1132D40EFD105E1012D36D0B6E07B2A27D1734CB3
S1132D5023680133022B01DC236000E02560704806
S1132D6001F0C2FD2368012B06D0022B07D0002BF3
S1132D700FD13020634904E03020634901E0634906
S1132D8030200522FFF7F6FDA02066490A22FFF74E
S1132D90F1FD612064217B2201F0DCFFC9E7062AF2
S1132DA006D14A4B60491878162201F07BFDC0E732
S1132DB0832ABED1BBE7B72A09D0DD2A02D07C2AF8
S1132DC063D109E031680829B3D13560B1E7281C23
S1132DD003F016FA55486CE0FF20FFF791FD041C40
S1132DE0820602D5524801F07FFDE30605D5E120B5
S1132DF0FFF786FD4F4801F077FD610640D54E4848
S1132E00240701F071FD6D460021600F01F074FD8F
S1132E100F354A4801F068FD0122291C6020FFF7A4
S1132E20D1FD2878082101F067FD2A78202A03D9EA
S1132E30E220FFF765FD23E004AC6120211CFFF7CD
S1132E40C1FD00272B789F4205DAE05D912101F056
S1132E505CFD0137F6E73A4801F046FD274B1B6855
S1132E60002B0DD12A78211C5208A820FFF782FDDF
S1132E7023782A780133A820211C2370FFF77AFDD8
S1132E8070212720FFF756FD53E7283AD2B2042ACF
S1132E9000D94EE72B4801F027FD2379292B07D0D1
S1132EA02A2B00D045E7281C03F0AAF9264800E0A5
S1132EB0264801F019FD3CE792B20198211C01F06B
S1132EC00FFA36E720FEFF1F1CFEFF1FF7FFFF1F50
S1132ED0A16B00000CFEFF1F212A0000152A000030
S1132EE02D2A00003480044003600740016007403D
S1132EF0006007400660074050F00F4018FEFF1FB7
S1132F00BE6B00009C6B0000656C0000346B00001D
S1132F1044F00F40CA6B0000D36B000014FEFF1F87
S1132F20DB6B0000396B0000436B0000E56B0000B5
S1132F30F76B0000066C0000136C00002D6C0000A1
S1132F40036C0000316C00004F6C00003A6C000010
S1132F50326837231A422AD0164E307801F0D0F95D
S1132F60002824D0144F3078211C402201F0B8F9F5
S1132F70051E1CD0201C291C00F07EF93A88201C58
S1132F80291C002A0FD101F049F80028EBD0802039
S1132F90400000F04DFA0228E5D1307807491722A5
S1132FA001F080FCDFE7002201F038F8DBE71DB018
S1132FB0F0BDC046F7FFFF1F30FEFF1F6A6C000024
S1132FC0F8B5274B80201A68C00002431A60254CCC
S1132FD0254A264922600D68402295430D601D68EC
S1132FE005431D60224D2560224D10242E68A64302
S1132FF02E600D68204E2C430C601C6880218900D3
S11330000C431C601D4D1E4C25603568202425434F
S113301035601C4D2F6827432F601F6838431860A4
S1133020C0271948BF0007601868D02708431860F4
S11330301648BF0007601868154F08431860154804
S113304007601868014319600020211C03F0ECF9A3
S11330503368234333602B681C432C60F8BDC0469F
S11330603880044080A004400301400054F00F4025
S11330700401100040F00F4000F00F400001200058
S11330808090044014F00F4000A004401C900440C1
S1133090030300001890044000B50A78031C002ABA
S11330A006D01B78013101309A42F6D000200CE0A2
S11330B000214156202907DC00229A56202A01D1FA
S11330C00133F9E7181C00E0101C00BD00B50368CB
S11330D000229A56202A05D020211A788A4301D04A
S11330E00133FAE700229A56202A01D10133F9E785
S11330F00360002018564342584100BD08B50548F6
S113310001F0F2FB044801F0EFFB044801F0ECFB92
S113311008BDC046F8700000F47900000B7100008F
S1133120F0B52C4A2C4E13780C2253439C59F318B7
S11331301A798BB0071C019203A820211B225D7908
S113314001F076FA002F04D0BD4210DD0C34013DAD
S1133150FAE7224801F0C8FB1E4A13780C225343B5
S1133160F618B06801F0C0FB1D4801F0BDFB1D4E10
S11331701D4F002D29D030780021422201F092FB0E
S1133180002808D130784021184A01F093F8184BF0
S113319001201D601CE0206801F0A6FB019B021CBD
S11331A030789A4202DB03A9012203E0019B03A9C0
S11331B09A1A92B201F076FB606801F095FB381C14
S11331C001F092FB0C34013DD3E7094B281C1D6030
S11331D00BB0F0BD3BFEFF1F747000000A710000CD
S11331E00E7100000CFEFF1F0B7100006D1000003B
S11331F02CFEFF1FF0B51D4E857B1D4F8BB002AC1E
S1133200281C211C052201F06BF800282BD0E37840
S11332102279012B02D0412B08D01EE0DD2AEED109
S113322030680028EBD0FFF77BFFE8E792B2281C58
S1133230211C01F055F82378042B08D1684669460F
S113324007300931012201F0FCF90A4802E0032B9E
S1133250D5D1381C01F048FBD1E792B2281C211CBF
S113326001F03EF8CBE70BB0F0BDC0462CFEFF1FCB
S1133270377100002671000008B50A1C0349031CBD
S11332800878191C01F00EFB08BDC046F7FFFF1FAC
S1133290F8B5204B051C1421186803F091FB1E4956
S11332A0071C03F08DFB2A1C0021041C01F0BCF850
S11332B0194D44216C434170612181707921C170A1
S11332C073213D1B20220171E1210270861D427190
S11332D00901281C03F074FB321C0021041C01F0BA
S11332E0A3F8E1231B015C433A262C1B471C067000
S11332F03C21201C03F064FB3A1C0221051C01F054
S113330093F80670421C3C2045430221601B01F0E7
S11333108BF8F8BDFCFEFF1F8051010038B50E4B41
S1133320021C1B689C78D87824029D79041958796A
S1133330D9792D021B79000428181B064018C018DF
S1133340022101F071F8A4B22D21421C0170201C4D
S11333500A2101F069F838BD1CFEFF1F7FB505483E
S113336001F0C2FA01A8FFF7D9FF01A801F0BCFAE5
S113337007B000BD517100007FB5031C02380B2853
S113338045D803F009FB0644114444443A35182552
S1133390182DFFF7E3FFFFF7B1FE1E4801F0A4FA72
S11333A01D4B1868393020E01B4B14221868393043
S11333B001F047F92BE00C3B581E83410220C01A50
S11333C001A902F0ABF901A801F08EFA13480CE050
S11333D0082002F0A3F9124801F086FA0C2013E049
S11333E00820002102F09AF90E4801F07DFA0EE05F
S11333F0042002F093F90C4803E0102002F08EF947
S11334000A4801F071FA0A200021FFF7B5FF07B05E
S113341000BDC046637100001CFEFF1F036C00006A
S11334207B7100008B7100009B710000AA71000089
S1133430802310B55B0098420BD1164B02241B88E5
S1133440002B25D1144B1B88002B21D1FFF702FB45
S113345003E08022104B92001A80104B1A888023BC
S11334605B009A4202D12020FFF7F4FAFFF776FFBF
S1133470FFF744FE0A4801F037FA0A4B00241868A3
S1133480393001F031FA084B201C1C70FFF748FE5C
S1133490201C10BD38FEFF1F24FEFF1F30FEFF1F3F
S11334A0637100001CFEFF1F3BFEFF1F00B53228A6
S11334B00FD0332819D0312824D1134B134A18685C
S11334C012681968124B10401B688B43184300059F
S11334D016E00D4B0D4A1868126819680C4B104021
S11334E01B688B43184340050AE0074B074A1868DA
S11334F012681968064B10401B688B4318438004FC
S1133500C00F00E0002000BD54F00F4040F00F4019
S113351050F00F4000B5322807D0332809D03128A5
S11335200DD1084B1B68DB0A06E0064B1B689B0A9F
S113353002E0044B1B685B0B0120984300E0002071
S113354000BDC04654F00F4038B5031C303B00208A
S1133550032B4FD8181C03F01FFA020A0508802415
S1133560240106E08024A40103E0002401E0802477
S1133570E4005DB264290BD003DC0020612939D05A
S113358003E0692904D06F291BD00120404231E0B7
S1133590194B80221968D2000A431A6001200322C1
S11335A0211C02F041FF154B1A68A2431A60144B08
S11335B01A680123AB4050321D1C1378AB431370BF
S11335C017E00D4B80221968D2000A431A60211CAF
S11335D00422012002F028FF084B1A6814431C60DF
S11335E0074B1A68012350321178AB401D1C0D4360
S11335F01570002038BDC0463880044054F00F4098
S11336001CFEFF1F00B5002905D0134B802219684A
S1133610D2000A431A60114B1968C20703D58022ED
S113362012010A4301E00E4A0A401A60196882072F
S113363003D58022D2000A4301E00A4A0A401A60F4
S11336401968420703D5802292010A4301E0064A21
S11336500A401A6000BDC0463880044040F00F4064
S1133660FFF7FFFFFFFBFFFFFFDFFFFF0F4B70B50F
S11336701B6801211A1C5032513316781878012422
S113368030401870FFF7BEFF30206921264200D079
S11336906F21451C49B240B26400EDB2FFF754FFFC
S11336A0E4B2382D01D0281CEFE770BD1CFEFF1FCB
S11336B070B52E4B041C1A7852B2002A30DB1A78EB
S11336C002210A422ED11878042210422CD11878F3
S11336D085062BD41E78012040251B78064203D092
S11336E02B4225D0224934E02B4223D1214B1D7893
S11336F0054221D11878084220D1197811421FD1EE
S11337001A7811071ED41A1C1B78DD061CD41378F2
S113371099061BD413785BB2002B19DA164918E00A
S1133720164916E0164914E0164912E0164910E04D
S113373016490EE016490CE016490AE0164908E05D
S1133740164906E0164904E0164902E0164900E06D
S11337501649002C04D1081C01F0C6F8201C04E012
S1133760201C01F006F9001BC0B270BD00F0074038
S1133770D76F000001F00740696D0000C76C0000BE
S1133780CC790000AC6D0000646F0000BD6F0000D8
S1133790306F00009C6C0000C06C0000606D000085
S11337A0B76D0000396F0000B9790000D36F0000D5
S11337B0F8B502F0D3FC164E164F051C0024601E0B
S11337C0072805D803F0E8F806080A0C0E101214AE
S11337D0301C0EE010480CE010480AE0104808E0E5
S11337E0104806E0104804E0104802E0104800E0E9
S11337F0381C01F079F8A54202D10E4801F074F8A2
S11338000D48013401F070F8092CD8D1F8BDC04638
S1133810B971000001720000C1710000CA7100009A
S1133820D3710000DC710000E5710000ED7100004F
S1133830F77100000B720000036C0000F0B50D1C62
S113384091B0161C072800D9CEE303F0AFF80800A6
S113385037003002CD03CD034D02B403B903081E73
S113386005D0042907D10122BB4B00201A70FFF7B1
S113387057FC041CC6E302220529F5D003220629BD
S1133880F2D004220729EFD005220929ECD0062220
S11338900A29E9D007220E29E6D008220F29E3D00D
S11338A009221029E0D00A221129DDD0002412298E
S11338B000D0A7E3A84B201C1C70D8E70592202950
S11338C000D991E3081C03F071F821003400C00012
S11338D08F03AB0073008F038F038F038F03540098
S11338E05E008F038F038F03D7009F019F018F0317
S11338F08F038F038F038F038F038F038F032400A2
S11339008F038F038F038F032B002E0002F0E0FC44
S11339106AE3924800F0E8FF0020FFF7C9FE63E382
S1133920FFF746FF60E300201056303802F068FCD1
S11339305AE38B4800F0D8FF8A4800F0D5FF8A4844
S113394000F0D2FF01F090F8822100F0DEFF8748FA
S113395000F0CAFF01F07CF8822100F0D6FF844811
S113396000F0C2FF01F066F8822100F0CEFF81482A
S113397038E306A8FFF78CFC002404707E4800F0AE
S1133980B3FF06A85EE01378313BDBB2032B01D909
S11339907A4827E37A4800F0A7FF059900200856E3
S11339A0FFF7B8FD041E01D176484BE0764819E3D1
S11339B01078031C313BDBB2032B01D9734811E3AC
S11339C040B2FFF7A7FD041E01D071480AE3051CAD
S11339D001263120471C40B2FFB2FFF767FD0028E3
S11339E001D03543EDB27600F6B2352F01D0F8B2EE
S11339F0F0E7059800F0DBFDC6B20598013E01230F
S1133A00B34001301E1C059000F0D1FD012801D106
S1133A10354300E0B543E8B20021FFF7F3FDF1E2DE
S1133A201378313BDBB2032BC8D85A4800F05CFF53
S1133A30059A00201056FFF739FD041E01D05648A0
S1133A40D0E2564800F050FFDCE2101C069200F071
S1133A50AEFD041C06A8FFF739FB002801D050482E
S1133A60C0E2069B2F34002160B25956FFF76CFD6B
S1133A70002800D1B8E2F2E70023D356002B01D18D
S1133A80102727E0101C00F092FD464B186005A893
S1133A90FFF71CFB059B1A78002AF1D020218A43EA
S1133AA052B204214C2A02D0572A04D102213E4AA0
S1133AB00133116005E0422A04D13B4A012111601F
S1133AC05B18059305980023C356002BD8D000F04B
S1133AD08AFD071C354800F007FF06AB2022314D54
S1133AE01A705A70002F00DC7EE28421286800F0EE
S1133AF00CFF2F4800F0F8FE6C4610211A34019197
S1133B00294A013F1368022B09D0042B0CD0012B46
S1133B1000D069E22B6811211E78301C08E0296866
S1133B200E881221301C03E02B6814211E68301CFF
S1133B3000F0EBFE1C4A296813685A182A60019A9F
S1133B40D21A0192022B35D0191F48424141182242
S1133B5049420A402FE0C0463BFEFF1F1572000099
S1133B602972000011710000407200004D720000C3
S1133B70547200000B710000667200008B7200002A
S1133B809D720000B0720000B9720000C1720000A2
S1133B90D0720000E0720000ED720000F1720000CB
S1133BA0F572000034FEFF1F04FEFF1FFD720000CB
S1133BB00E7300000822E118201C02910299884229
S1133BC012D0311CD1408C462039C9B203912E2128
S1133BD0009103995A2902D86146C9B2009100990B
S1133BE0083A01700130E9E7E418002F02D0019A85
S1133BF0002A85D10D2323700A2363700023A37048
S1133C0006A800F071FE6DE70023D356002B00D107
S1133C10EAE1101C00F0CBFC041C112D01D1BD48BD
S1133C2000E0BD4800F060FE05A8FFF74FFA059BD1
S1133C301A78002A00D1D7E120218A4352B2B74E24
S1133C404C2A01D1042202E0572A03D10222326015
S1133C50013304E0422A03D1012232609B18059308
S1133C6005A8FFF733FA059800F0A1FC071C05A886
S1133C70FFF72CFA0120112D07D1059B00229A563B
S1133C80002A02D0181C00F0AEFC3368002800DCC7
S1133C90AAE1022B05D0042B05D0012B04D12770F7
S1133CA002E0278000E02760E4180138EEE70029ED
S1133CB009D0032900D097E1994B101C1C6800F02F
S1133CC092FC208490E1974C2388042B05D19648DC
S1133CD000F00AFE1023238004E0944B081C198092
S1133CE0FEF7B8FE2C1C8DE1162900D97CE1081CD6
S1133CF002F05CFE17005F002B0041007C007A019B
S1133D007A017A017A017A017A017A017A017A01D7
S1133D107A017A017A019A007A017A017A014A01D8
S1133D204A017F4B824F1D680024E000001B3818B5
S1133D30311C00F004FE002802D10535EC7736E191
S1133D4001340C2CF1D17B484CE10023D356372BA2
S1133D5005D1734B01221B68D9690A4307E0382B4C
S1133D6007D16F4B01221B68D96991430A1CDA61A0
S1133D701DE1714836E16A4B704F1D680024A000B4
S1133D8000193818311C00F0DAFD00280CD1EA695A
S1133D9006239A43131C002C04D0012C00D01FE1ED
S1133DA002223AE0042238E00134032CE7D16448CB
S1133DB018E15B4B634F1D680024A0003818311CC8
S1133DC000F0BDFD00280CD1E969182399430B1CB0
S1133DD0012C04D0022C00D002E110221DE00822A4
S1133DE01BE00134032CE8D15748FBE04C4B574F00
S1133DF01D680024E0003818311C00F0A0FD0028E4
S1133E000DD1EA6960239A43131C012C04D0022CBF
S1133E1000D0E5E0202200E040221343E0E001343A
S1133E20032CE7D14A48DDE04A4800F05DFD4A48EA
S1133E3000F05AFD3A4C23680533DB7F0B2B04D882
S1133E40D800C31A3A48C01800E0444800F04CFDBA
S1133E50434D281C00F048FD23682E1CDB69D9075C
S1133E6001D5404800E0404800F03EFD3F4800F0E6
S1133E703BFD2368DA690123910704D404231A4023
S1133E80534253415B009800C3182C48C01800F0FB
S1133E902BFD374800F028FD23680220DB69DA0691
S1133EA001D41807C00F274B8000181800F01CFD20
S1133EB0304800F019FD23680125DB69590602D456
S1133EC09D06ED0F6D002C4800F00EFD1F48EB0021
S1133ED0C01800F009FD301C00F006FD002D00D1D3
S1133EE082E0264800F000FD236800214E33187854
S1133EF000F002FD224D281C00F0F6FC214800F0E1
S1133F00F3FC236800214F33187800F0F5FC281CDB
S1133F1068E0C046137300001A73000008FEFF1F18
S1133F201CFEFF1F24FEFF1F2273000038FEFF1F2C
S1133F30696F0000D67300002E730000C46F000088
S1133F40EF730000546D0000027400005C70000008
S1133F5018740000467300005F730000677300006C
S1133F60036C00007073000072730000747300002F
S1133F70F87300007C7300008B73000099730000D9
S1133F80A5730000A9730000101C00F02CFBC0B244
S1133F90632803D8002802D1012000E063201B4BD2
S1133FA01B68152D01D14E3300E04F3318700420E7
S1133FB0FEF7ACFD18E0081C111CFFF7DDF913E057
S1133FC0062911D11248111C00F0B9FC041E0DD0B1
S1133FD01048311C00F0B3FC041E0DD00E4801E063
S1133FE0EB61E4E700F080FC00240BE0074B402188
S1133FF01B685A8C0A4304E0044B40211B685A8C0A
S11340008A435A84201C11B0F0BDC0461CFEFF1F19
S1134010B4730000BB730000C3730000F0B587B035
S113402005910021071C04920391059B002B00D1EC
S113403001E13B78082B0DD1804B1A78002A05D07A
S11340407F48013A01301A7000F04EFC7D4A00238B
S11340501370EBE01B2B01D17A4905E05B2B06D1F1
S113406078490A781B2A02D10B700137DEE07549C2
S11340700A785B2A4FD1181C413803284BD802F028
S11340808BFC101009026D4B1A78002A00D1CDE088
S1134090013ACAE0694B1A78272A00D9C6E00132EE
S11340A0C3E0694C28202268684D5043281800F06A
S11340B06CFC3B78061C412B08D12368002B01D1F2
S11340C0032300E0013B2360614806E023680133D9
S11340D0032B00DD00235F48236000F005FC351C42
S11340E05D4E002D04D0301C00F0FEFB013DF8E7CE
S11340F0584800F0F9FB206828256843534B1818EA
S113410000F0F2FB206851494543481900F03DFC9A
S11341104A4B18708AE00A2B00D187E0002B00D1AB
S113412084E0494A28251268444C02920299227874
S11341306943464E89188B553B780D2B6AD10A2367
S113414004988B55FEF7C6FC3F4B444A1B68127813
S11341500C205D4342432378414901337519545877
S1134160DBB28A185679EA180021013A11700499D1
S1134170002905D13B4A1288002A39D0510537D489
S1134180002B32D0281C002E19D02168FEF784FFA2
S1134190013E0390002810D0334800F0A5FB207A9C
S11341A0617A039AFFF74AFB002802D12F4800F0F6
S11341B09BFB049A002A1BD112E00C34E2E72C4941
S11341C0FEF76AFF021E10D004200921FFF736FB18
S11341D0002802D1254800F087FB049B002B07D15F
S11341E0204B1888FEF736FC02E0224800F07CFBE6
S11341F0FEF782FC114B00221A70134B196801312F
S1134200032903DC19600121039105E01A600122EE
S1134210039201E0013222700A4B00221A70074B0C
S113422001371A78272A01D927221A70059B013BE6
S11342309BB20593F9E6039807B0F0BD3AFEFF1F61
S1134240A16C0000DCFEFF1F28FEFF1F3CFEFF1FC9
S1134250317400000C710000117300003BFEFF1F5D
S11342607470000030FEFF1F036C0000F972000040
S113427035740000F572000013B5441E0548E4B21D
S113428000682301C318187B00941C680323A0470B
S113429016BDC046E0FEFF1F08B5044B18700001B0
S11342A000F0A4FB024B186008BDC046DDFEFF1FF2
S11342B0E0FEFF1F37B5031C0D1C0020FF2B0CD0A4
S11342C00648013BDBB2046819016418207B0093A3
S11342D0111C24682A1C0223A0473EBDE0FEFF1FD8
S11342E013B5441E0548E4B200682301C318187BC3
S11342F000941C680423A04716BDC046E0FEFF1FBF
S113430013B50749421E0968D2B21301CB18187BB2
S1134310002100921C680A1C0523A04716BDC04654
S1134320E0FEFF1F30B50A4B0A4A1B6814780022CE
S1134330A2420BD01D680132854204D11D7B8D42FF
S113434001D1D0B203E0D2B21033F1E7002030BD86
S1134350E0FEFF1FDDFEFF1FF0B5061C85B0101C3C
S1134360019102920393FFF7DDFF011E01D00020AB
S11343703AE0FFF7D7FF071EF9D01C4BC5181C4BBA
S11343802D011B685D193388002B13D0039800F0AE
S11343902DFB041C68600DD03388181C009300F0BA
S11343A025FB0028E3D0009B20606060A060C0185B
S11343B0E060E3827388002B11D0039800F016FBB1
S11343C0041CA8600BD07688301C00F00FFB00287A
S11343D0CDD020606060A0608019E060E682029B1E
S11343E0381C2B60019B2B7305B0F0BDFFFFFF0F42
S11343F0E0FEFF1F07B500280ED0002103280FD1CF
S1134400108901AB1268188059801178181C054A6C
S11344101823FFF7A1FF04E0101C00F0C1FE00E028
S1134420081C0EBDC9460000F0B50E1C85B0141C56
S1134430CB0604D52023137004239E430134F307D1
S113444006D5002804DA2D2323704742013400E006
S1134450071C00230193022333402F4D0393002FA5
S11344602DD0BD4214D9281C0A2102F0A9FA019BBF
S1134470051C002B04D10128F3D1039B002B01D090
S1134480302302E07307ECD5202323700134E8E7DE
S1134490002D01D001230193291C381C02F090FA4D
S11344A0631C0293031CC0B26843303323703F1A69
S11344B00A21281C02F084FA029C051CCFE730274D
S11344C0201C019B002D09D0002B09D0281C0A2197
S11344D002F076FA2770051C0134F1E7002B0DD1A8
S11344E0730703D52023601C237007E0B30702D5AC
S11344F03023601C2370302303700130330704D54C
S11345000D2303700A234370023040231E4000D160
S1134510067005B0F0BDC04600CA9A3BF7B5CB069D
S113452002D52023137001324BB2002B04DA30235E
S1134530137078235370023220230B400093082316
S11345400B404026019307230E4019400F1C0429F9
S113455000D90427FFB27F000F21141C3B1C8C469A
S1134560013BDBB2FF2B15D09D00011CE9400D1C63
S113457061460D40291C3031392908D90099002998
S113458002D0291C373102E0291C5731C9B22170ED
S11345900134E5E7019BD019002B04D00D230370EF
S11345A00A2343700230002E00D10670FEBD10B500
S11345B0031C00229A56202A01D10133F9E7002076
S11345C00F241A7851B22F290CDDD1B20A1C303ACB
S11345D0D2B200010133092A02D90A1C573A2240F7
S11345E01043EEE710BD10B500220378191C3039D2
S11345F0C9B2092906D9002B18D02D2B00D10122CC
S11346000130F2E7002301780C1C303CE4B2092CA1
S113461007D85C00303CDB00E31849B201305B187A
S1134620F1E7181C002A02D0584200E0181C10BD03
S113463000B5031C8218934202D019700133FAE7C3
S113464000BD10B50023934203D0CC5CC4540133A5
S1134650F9E710BDF7B5038A041C0E1C4768151C46
S11346609A4200D91D1CADB2002D28D0E3687A19F6
S113467062609A4215D3DB1B9BB22268E91A00934D
S113468053186360019101F09DFA002E12D0391C79
S1134690009A301CFFF7D5FF009B2168F018019A9F
S11346A006E001F08FFA002E04D0301C391C2A1CBD
S11346B0FFF7C7FF01F07EFA238A5B1B238201F018
S11346C081FA281CFEBD0000F8B51D1C06AB0F1CAA
S11346D0161C1C7801F06EFA052D0DD0062D12D093
S11346E0042D1BD1104B24011B68391C1C19606854
S11346F0321CFFF7AFFF15E00B4B24011B681C199C
S113470063681C8A0BE0084B24011B681C1963684E
S113471000241A681C829A605A6000E0002401F0A8
S113472051FA201CF8BDC046E0FEFF1FF7B5041C7B
S1134730151C0F1C01F03EFA218A628AE38A88184C
S11347404019984202DD5D1AAD1AADB2A168AA18EB
S1134750628201914A19E168A2602E1C8A4205D343
S1134760D31A2268A3609B1AEE1AB6B201F02AFA91
S11347700198391C321CFFF764FFB54204D0B91903
S1134780AA1B2068FFF75DFF01F014FA638AA28A6E
S1134790AB4206D1238AEB189A1800232282A38203
S11347A002E0AA18A2825B1B638201F00BFA281CA8
S11347B0FEBD0000F7B5041C0191002936D1027832
S11347C043780D1C9A4261D101F0F4F9A178304B81
S11347D030481970FFF7A6FD2F49087000280ED045
S11347E02E4A2F4B80181B68000118184368207943
S11347F01A8A561D3618D88A864203DD0D7001F0D8
S1134800E1F943E006321A82A11D8C420CD09A6869
S1134810501C9860207810709868DA68904201D330
S1134820186898600134F0E706252FE01A4B1E78CB
S1134830002E0DD102784378351C9A4226D1877810
S11348401448391CFFF76EFDFFB2061E06D11DE0A9
S11348500F4A177800221A7001F0B4F90F4A104B6E
S1134860B6181B6836019E19E3787068032B04D1CF
S1134870C58A038AED1AADB208E0211C019AFFF73C
S113488055FF0421051C78B200F02EFA281CFEBD49
S1134890E5FEFF1FC9460000E4FEFF1FFFFFFF0FF8
S11348A0E0FEFF1F08B5031E04D1081C111CFFF70E
S11348B081FF05E00020FF2B02D0181CFFF7DCFC71
S11348C008BD38B5041C031C1A1B0133581E057897
S11348D092B2002DF8D1281C002A03D0081C211CF8
S11348E0FFF7E0FF38BD000008B5024B1978FFF769
S11348F0E8FF08BD0CFEFF1F1FB56A46FFF794FDD5
S11349006846FFF7F1FF05B000BD1FB56A46FFF723
S113491005FE6846FFF7E8FF05B000BD07B5031CB8
S1134920002083420AD06A4610705070937011714F
S1134930012368460521D370FFF73CFF0EBD00B587
S11349400378002B0FD000228A565BB2934207D023
S1134950D80FD1179A42484140420123184307E037
S113496001300131ECE700200856431E98414042D3
S113497000BD10B5031C0C78181C1C700A78013398
S113498052B20131002AF6D110BD00B5021C031C3D
S1134990981A0133591E097849B20029F8D100BD8B
S11349A00E4B13B500221A800D4B0E4A19600E4BA4
S11349B0147819601A1C0378A34203D0002B0CD07E
S11349C00430F8E74388C9186B4611600733552251
S11349D0994202D80A700131FAE713BDECFEFF1FB9
S11349E0E8FEFF1F12FEFF1FF0FEFF1FF8B50E4F7B
S11349F00E4E3B683488051C1C1903231C4201D04D
S1134A009C4304340A4A631912689A420AD92A1C3C
S1134A10201C0021FFF70CFE3B68201CE31AED1854
S1134A20358000E00020F8BDE8FEFF1FECFEFF1F0C
S1134A30F0FEFF1F054B00B51A68131C981A0133CA
S1134A40197880B25529F9D000BDC046F0FEFF1F89
S1134A50034B1868034B1B68C01A80B27047C046EA
S1134A60F0FEFF1FE8FEFF1F044B1868044B1B6891
S1134A70C01A044B1B88C01A80B27047F0FEFF1F97
S1134A80E8FEFF1FECFEFF1FF0B585B00392574F01
S1134A90574A002313603B60564B061C1B780C1CC2
S1134AA02578002D48D06DB29D423ED1221CA31A18
S1134AB0DBB20293013400256557002DF7D1142091
S1134AC058430430FFF792FF02993860CB43E4184F
S1134AD02F1C6178002926D049B2331C01911A6831
S1134AE0002A1ED0002151568C4601998C4516D1BE
S1134AF05968026041601A890281002A01D0013597
S1134B00EDB2598941819A8982819B7BC3730029C3
S1134B1001D1002A01D00137FFB2143001E0103373
S1134B20DDE70134D5E7016008E001340022A25634
S1134B30002AFAD10134B3E72F1C02952B4C2368C9
S1134B40002B47D0002F2BD00C207843043080B2A8
S1134B50FFF74CFF264E284A2368306094461A68B3
S1134B60002A19D05A89002A06D0624501D10021B1
S1134B7059815A89426003E09989002901D0416032
S1134B8001224168002901D001214172002A01D08B
S1134B9003600C301433E2E70C235F43C01B306026
S1134BA0039BE818C0B2FFF777FB002D12D02468EE
S1134BB0216800290ED02389002B09D0032001216C
S1134BC0221CFFF717FCA073002801D1FF23A37355
S1134BD01434EDE7094800F0C5FF094B00221A60C0
S1134BE001F0EAF8029805B0F0BDC046F4FEFF1FDC
S1134BF000FFFF1F12FEFF1FFFFF0000F8FEFF1F54
S1134C00FCFEFF1F054A06481188CB07DB1703404B
S1134C1049084B4098B210807047C046F8FEFF1F09
S1134C2000B4FFFF184B37B51C682368002B29D04C
S1134C30E27B0D231A4223D000F0BCFFA389002B92
S1134C4002D1E37BD90716D4237C002B0ED0002598
S1134C506A46157055702168281C0A7869468A705E
S1134C600522CD700B71FFF71DFE2574E27B0A232C
S1134C70134000D1E37300F0A5FF201C6268904745
S1134C801434D2E737BDC046F4FEFF1F38B50C4BD1
S1134C90051C1C6800F08EFF0D222368002B0CD02D
S1134CA0E17B114207D01B785BB2AB4203D000F02A
S1134CB089FF012002E01434EFE7181C38BDC04618
S1134CC0F4FEFF1F00B5074B1B681A68002A07D0C3
S1134CD0127852B2824201D1D87B02E01433F4E755
S1134CE0802000BDF4FEFF1F38B5174B1C682368F5
S1134CF0002B27D01B785BB2834221D1002918D125
S1134D00124B1D68002D14D02B68002B11D09C422F
S1134D100DD100F04FFFA389002B03D00C4A126879
S1134D209B186B600023E37300F04CFF0AE00C3522
S1134D30EAE74A0702D5E37B1A0703D4E17301E0EB
S1134D401434D4E738BDC046F4FEFF1F00FFFF1F34
S1134D50FCFEFF1FF8B5194B0E1C1C68171C002C19
S1134D602BD0174B1D682B68002B26D01B785BB209
S1134D70834220D12368002B1FD09D4219D100F01B
S1134D8019FFEB7B02229343EB732772002F04D1AC
S1134D90AE81002E04D1667208E0002E00D10126F7
S1134DA0084B1B68F61801236660637200F00AFF63
S1134DB003E00C34DEE71435D5E7F8BD00FFFF1F30
S1134DC0F4FEFF1FFCFEFF1F38B5114B1D68002DBC
S1134DD01DD0104B1C682368002B18D01B785BB2C5
S1134DE0834212D12B68002B11D09C420BD100F0CE
S1134DF0E1FE00232B726B72E37B02221343E37305
S1134E0000F0E0FE03E00C35ECE71434E3E738BDD2
S1134E1000FFFF1FF4FEFF1F144A154B11681B68A7
S1134E200131F0B5101C1160002B1ED0022408259E
S1134E3004261A68002A18D0597A002913D0016868
S1134E405F68B9420FD1D17B214204D1294200D1FC
S1134E50D673197A11749289002A03D059688A1872
S1134E605A6000E05A720C33E3E7F0BDFCFEFF1F0A
S1134E7000FFFF1FF0B50D1C2C352B7885B0061CE8
S1134E800C1C9A070FD01121DA0700D4132101F06A
S1134E9069F8C0B2002861D12B78032293434022E1
S1134EA013432B705AE020271F4054D1088B00284D
S1134EB003D1402293432B704DE0CA681178A26A53
S1134EC0520516D50422134202D093432B7010E0EE
S1134ED0221C2E3212780192914205D02D22125DAD
S1134EE08A4206D1012804D004210B4301992B7076
S1134EF00127301C01F036F8236840220133236077
S1134F002B7813432B70002F28D1E3686269013397
S1134F10E360934201D3A368E360228B104B013A10
S1134F20B600F35892B222832F34998C2378002B45
S1134F3014D08A4212D86A46937201230025D37290
S1134F40DD23157255721373281C02A90522FFF77D
S1134F50A9FC257002E0301C00F0F4FF05B0F0BDA0
S1134F6008FFFF1FF7B5019308AB061C0D1C141CAA
S1134F701F7800F01FFE01980238082800D9EDE0E0
S1134F8001F00AFD05486E3BC2ECECEC9D00764B4B
S1134F903F011B68DF19E90401D5BF6800E07F68A1
S1134FA0002C28D0E20703D5301C00F09DFF04E05C
S1134FB0A30702D5301C00F0BBFF610703D5301CEA
S1134FC000F064FF04E0220702D5301C00F082FFE9
S1134FD0BB6AE10603D580225201134303E0A20613
S1134FE002D5624A1340BB62630604D57F231D4089
S1134FF03B1C2F331D703D8DB1E05B4B3F011B68A3
S11350005B4ADF197B689C6A144201D01D8CA6E0C0
S11350101D8BA4E0544B3F011B68DF19BF68002DB2
S113502007D1FA8B3B8BD31A9DB2A34200DB96E0E7
S113503094E000F0C7FD381C291C221C0830FFF73F
S113504075FB051C00F0B6FD3B1C2C331A7860235D
S11350501A4200D083E0301C391CFFF70BFF7EE0BE
S113506041493F0109680197CB195F68291C381C25
S1135070221C0830FFF7EEFABB6A6022051C1342BB
S11350806FD03A1C2C3211781020014269D03C8B2D
S1135090A446BC8CA44564D881431170990660D59C
S11350A0314C01202768019C3F19B9680B1C2C3333
S11350B01A7802431A70301CFFF7DCFE51E02A4BC9
S11350C03F011B68DF19012C05D9023CBB68A4B25F
S11350D0002D10D103E07B68002D0CD107E0012CDA
S11350E005D91D605D607B681D605D6037E0A400CC
S11350F00025E55033E0A4001C190023E25CEA54C7
S11351000133042BFAD129E0174D3F01002C03D0C1
S11351102B68DF19BB681AE029681024CA19536880
S1135120191C2C310878204211D0A04308709168D2
S11351308A6A920608D50B1C2C331A780120024384
S11351401A70301CFFF796FE2B68DF197B689A688B
S113515000251A61DA601D831D8400E0002500F03B
S113516031FD281CFEBDC046E0FEFF1FFFEFFFFF20
S11351708080000038B5051C3020FFF737FC041E82
S113518001D100200BE0281CFFF730FCA0600028B0
S1135190F7D043192061E0606361E583201C38BDCA
S11351A0F7B53E4E0091017A041C301CFFF7BAF8A3
S11351B0051C071C002D03D0009A520707D46BE08E
S11351C0291CFFF7AFF8051C381C002D64D0344BA4
S11351D0009AEF18334B3F011B68DF193E609207BA
S11351E007D5E088267AFFF7C5FF2F4BB600985104
S11351F0B860009A2D4ED20706D5A088FFF7BAFFF3
S1135200237A78609B00F050237A274A9B00D35876
S1135210002B0ED0226864219A62237A224A9B00D2
S1135220D358E0880093A37B584301F017FC009BFC
S11352309884237A9B00F358002B26D0227B2F33AB
S11352401A70237AA288607B9B00F3585043642130
S11352500092019301F002FC019B009A5884237A86
S1135260A07B9B00F35850436421019301F0F6FBAB
S1135270019B22689884237A9B00F3589A62237ACC
S1135280A27A9B00F3582E331A70237A211C3B73A5
S1135290207A00F0BBFD281CFEBDC046654F00000F
S11352A0FFFFFF0FE0FEFF1F08FFFF1F04FFFF1FAC
S11352B0F7B55B4A8B009C585A4A80279D58A36ACD
S11352C03F01061C01911F4014D0221C2C3211787E
S11352D004200F1C0740BC4603D0814311700027F3
S11352E010E0271C2E373F78B74202D101431170DA
S11352F094E067461A0605D5221C2D321778BF1B89
S11353007A4257412022134218D0132E08D12B1C65
S11353102C3319780A431A706B6801336B607DE093
S1135320112E0BD12B1C2C331978114276D09143BA
S113533019700198291CFFF79DFD6FE02268013266
S11353402260D9041AD52A8BEB8B9A420CD82A698D
S113535016702B69696901332B618B4201D3AA68EA
S11353602A612B8B01332B832B1C2C331A7860235B
S11353701A4203D10198291CFFF77CFD238BE28B91
S1135380002F32D19A420BD90133238323691E7033
S11353902369676901332361BB4201D3A168216199
S11353A0A36A602213421BD0261C2C363278D706FF
S11353B016D4218B628C914212D3990609D52B1CE9
S11353C02C331A7802210A431A700198291CFFF71A
S11353D051FD3378102213433370636801336360E3
S11353E0114BA26A1A4211D018E0218C0131218498
S11353F09A420BD90133238323691E702369676999
S113540001332361BB4201D3A16821612F34207889
S1135410002803D040B20421FFF766FCF7BDC04664
S113542004FFFF1F08FFFF1F8080000008B5034B27
S11354308200D158FFF71EFD08BDC04608FFFF1FBC
S113544008B500F0A1FB08BD08B56120B721FFF73E
S113545065FA08BDF8B53D4B3D4E1A68041C01328F
S11354601A6033780D1C0133DBB233703B2B4CD9FB
S1135470384F3B780133DBB23B703B2B38D9364B8A
S11354801A780132D2B21A70172A24D900221A705B
S1135490324A3348117803780131C9B211700133AB
S11354A0DBB2062B01D9073BFAE703701D2907D1AC
S11354B02C4B1978022903D10121117003221A708F
S11354C02A0708D5E368002B05D000F073FBE268D7
S11354D0904700F077FBAB0608D56269002A05D037
S11354E000F068FB6369984700F06CFB00233B7095
S11354F0AA0708D56368002B05D000F05BFB62683F
S1135500904700F05FFB00233370EB0508D5A268D9
S1135510002A05D000F04EFBA368984700F052FB28
S1135520AA0508D52368002B05D000F043FB2268A8
S1135530904700F047FB2369002B05D000F03AFBAD
S11355402369984700F03EFBF8BDC0460CFFFF1FDF
S113555011FFFF1F12FFFF1F10FFFF1F0EFEFF1F93
S11355600DFEFF1F0FFEFF1F0D4B1B78C3720D4B6B
S11355701B8883800C4B1B7883710C4B1B78C37185
S11355800B4B1B7803720B4B1B7843720A4B1B7833
S113559083720A4B1B680361802303737047C04600
S11355A011FFFF1F10FEFF1F0FFEFF1F0EFEFF1F48
S11355B00DFEFF1F10FFFF1F12FFFF1F0CFFFF1F39
S11355C0F0B5002801D1414B1960414A414E424F88
S11355D004230325541EA4B22C420CD1B9420ED983
S11355E03E4C02330919DBB2062B02D8013292B2C7
S11355F0F0E7073BF7E7B14206D8002500E00125B4
S1135600374E0022B44608E0364C01330919DBB2A8
S1135610062BEBD9073BFAE70222002D0BD0012A17
S113562009D1614517D9304E1D338919DBB2062BD8
S1135630F2D9073BFAE72D4FBE5C2D4F7743B942B1
S113564009D9C91BF318DBB2062B01D9073BFAE7CA
S11356500132D2B2E1E70132254DD2B20127A9428B
S113566009D9244E01378919FFB20133DBB2062B65
S1135670F5D9073BFAE7204E0025B446614504D925
S11356801E4E01358919EDB2F8E700263B2903D9EE
S113569001363C39F6B2F9E7C9B2002807D0827165
S11356A0C7710372C1728672457284800DE014481A
S11356B00270144A1770144A1370144B1970144B67
S11356C01E70144B1D70144B1C80F0BD0CFFFF1F8B
S11356D0B30700008033E1010085E201007B1DFE79
S11356E0803B260080CC1EFE80C4D9FFFD790000DB
S11356F08051010080AEFEFF0F0E0000F0F1FFFFAD
S11357000FFEFF1F0EFEFF1F0DFEFF1F11FFFF1FE9
S113571012FFFF1F10FFFF1F10FEFF1FF0B58BB01D
S113572005AD061C0C1C281C0021142201F0F8F9FC
S1135730022E0FD10B232B73002C0ED0281C00F04B
S11357402BFCAA88704B9A4207D8201C6F49FFF79C
S113575010F92DE0281CFFF707FF032737402AD054
S1135760002C24D0221CE8790021FEF75DFE3A26A5
S11357700670421C0221A879FEF756FE0670421CF0
S11357800021A888FEF750FE1221021C687AFEF759
S11357904BFE0670421C0221A87AFEF745FE021C4D
S11357A00670E87A01320221FEF73EFE00E0201C7A
S11357B0001BC0B2A6E0002C00D195E0082E0AD14F
S11357C00023E3562B2B09D101340023E356202B6D
S11357D0FAD0012702E0182E00D10826201CFEF77B
S11357E002FF0290C0B2039023781A1C303AD2B25E
S11357F0092A01D80134F7E7002101918B4210D026
S11358000134201CFEF7EFFEC0B201902378303B38
S1135810DBB2092B01D80134F8E73B1C5A1E934133
S1135820FF180022A25600239A4208D00134201CFB
S1135830FEF7D9FE3A1C511E8A4183B2BF18082EC6
S113584011D12278111C3039C9B2092901D8013487
S1135850F7E7211C202A06D14A780134303AD2B223
S1135860092A00D81826F2060CD503980199264A6D
S1135870E871A971AB80934233D8FA22D2009B1805
S1135880AB802EE0032F26D8381C01F085F80208DF
S11358900C15039801996872A972EB7221E0029ABF
S11358A02869D3B206E002993C22CBB253432A6959
S11358B001989B181B180CE0029A2869D1B2E122C6
S11358C012014A43121801983C214143DBB2521899
S11358D0D3182B6101E0002F03D0281C2969FFF79E
S11358E06FFE182E00D178E7082E04D1084B0593DB
S11358F006232B7302E0012205AB1A73281C00F067
S11359004BFB00200BB0F0BDCF070000097A00006C
S113591049540000F0B585B00391818804220291B6
S1135920364900230324029DA94214D24D1C21426E
S113593007D1334F0232DB19D2B2062A09D9073A0A
S1135940FAE7304901325B18D2B2062A01D9073A84
S1135950FAE7291CE7E78779032421408C462A4D7E
S1135960391C2A4E0197013900290AD001394C5DAE
S1135970371C6743A218DB19D2B2062AF4D9073AB6
S1135980FAE7614600290AD1019D022D07D91F4F6C
S11359900132DB19D2B2062A01D9073AFAE7C679ED
S11359A0771ED219D2B2062A01D9073AFAE7457A04
S11359B0847AC17AE1200001684384463C20604334
S11359C0604440180090114847430098C719F818DC
S11359D0039B002B0FD00E4B029F1F800D4B019F8A
S11359E01F700D4B1E700D4B1D700D4B1C700D4B1D
S11359F019700D4B1A7005B0F0BDC046B207000017
S1135A000085E2018033E101FD790000805101004D
S1135A1010FEFF1F0FFEFF1F0EFEFF1F10FFFF1FD4
S1135A2012FFFF1F11FFFF1F0DFEFF1F10B586B0F1
S1135A30041C422301A80373019400F0ADFA021E72
S1135A40012A05D1034B6B2014211C60FFF782F956
S1135A5006B010BD14FFFF1F30B50B4D847B89B019
S1135A60201C69460522FEF73BFC00280AD06A4642
S1135A70D378002BF4D11379012BF1D12868FFF7E7
S1135A80D5FFEDE709B030BD14FFFF1F08B56C204A
S1135A90FFF7FCF8002801D100F04AFB08BD70476D
S1135AA0704770477047704770477047704770473A
S1135AB00C4A10B513680C4C002B0AD0013B136040
S1135AC0002B06D12368DA0703D580229200134302
S1135AD0236006482168FFF7BDFC2268044B13408D
S1135AE0236010BD98FFFF1FDCFFFF1F9CFFFF1FFB
S1135AF0FFFEFFFF70B5154D154C2B6822681A4048
S1135B0091020BD5134A144E1078336800211840C3
S1135B10FFF7CEFB2B681A0300D5326822681340C6
S1135B20190202D50020FFF781FC2A682168084B7E
S1135B300A40510208D51968084A0A401A60084BFD
S1135B40012219689143196070BDC04604400540A4
S1135B5008400540F6FFFF1F0C400540FFFFBFFF54
S1135B60E0FFFF1F054B10B51C682388002B00D1F4
S1135B70034B0380FFF746F8208010BDB8000020D7
S1135B807B12000070470000074B00B51A680C2315
S1135B901A4204D0054B55221A60AA221A60044BFB
S1135BA0802212011A6000BD008104400481044077
S1135BB04CF00F4072B6024B1A6801321A607047FB
S1135BC0D8FFFF1F044A00B51368013B1360002B84
S1135BD000D162B600BDC046D8FFFF1F08B5054B13
S1135BE01A681A60FFF7E6FFFFF716F9FFF7EAFFF6
S1135BF008BDC0460000044010B5074B074C002206
S1135C001A60A368934205D0FFF7D4FFA3689847AE
S1135C10FFF7D8FF10BDC04608D003409CFFFF1F0C
S1135C200268802310B51A421CD0144A4C00A25AB0
S1135C30D40403D51205120D026013E00360012998
S1135C4006D0022909D000290CD10D4B0D4A06E0DB
S1135C500B4B0D4A1C68224003E0094B0B4A1868A1
S1135C6002401A600A4B8900CC58002C04D0FFF77C
S1135C70A1FFA047FFF7A6FF10BDC046F0FFFF1F1E
S1135C803C800440FFFFFFFEFFFFFFFDFFFFFFFB23
S1135C90E4FFFF1F08B502480221FFF7C1FF08BD5A
S1135CA000A0034008B502480121FFF7B9FF08BD71
S1135CB00090034008B502480021FFF7B1FF08BD7A
S1135CC000800340F7B5134B1C681F1C002C1FD029
S1135CD0114E1C6001252C4215D032680192FFF749
S1135CE069FF0E4A93190E4A9B181B689847019B3B
S1135CF0B02212031A4080231B039A4200D13D6054
S1135D00AC43FFF75FFF6D000436002CE3D1DAE704
S1135D10F7BDC046A0A0044000A0044018FFFF1F28
S1135D200060FBBFF8B5124B1C78E4B2002C1ED007
S1135D3000260125254215D00123AC43B340012B95
S1135D4004D0202B04D1FFF757FF01E0FFF746FFF3
S1135D50084AB3009F58002F04D0FFF72BFFB84721
S1135D60FFF730FF6D000136EDB2002CE2D1F8BD33
S1135D7004C00740B4FFFF1F0C4A89018318C9B24D
S1135D8000B51970C317DB0E1B18094A5B119B0081
S1135D909B18084A104004D520220138524210436F
S1135DA00130012282401A6000BDC04600E400E0D8
S1135DB000E100E01F0000800E4B0122196805205D
S1135DC0114319600C4B802119600C4908600C497F
S1135DD0C02008700B4980204005086019684020E5
S1135DE00143196008493120086019680A431A60A0
S1135DF07047C0463880044000000440040004405A
S1135E001CE400E000E100E00800044010B50028B4
S1135E1031D1194B80221868520302431A60174B80
S1135E2080221868D20402431A60CB7A9D200B2B7F
S1135E3002D8134A5B00985A0A68F0210905114BED
S1135E400843186006211048D40707D57F2404703E
S1135E50114008D00221500705D503E0FF24047047
S1135E60114000D003219960D00604D5196880221E
S1135E7092010A431A6010BD388004400480044033
S1135E801A7A000000400540F6FFFF1F00B5002805
S1135E900FD10B4B80221968D2000A431A60094BB8
S1135EA0802292001A60084B80221A70074B52011C
S1135EB01A60074B8022996812030A439A6000BD56
S1135EC03880044004A004400CE400E000E100E059
S1135ED000400540024B034A99680A409A607047A3
S1135EE000400540FFFF77FF00B500280FD10B4BA2
S1135EF080221968D2000A431A60094B802292005A
S1135F001A60084B80221A70074B52011A60074B23
S1135F109022996892030A439A6000BD3880044035
S1135F2008A004400CE400E000E100E0004005406B
S1135F30024B034A99680A409A6070470040054042
S1135F40FFFFDBFF054B80229968D2030A439A6066
S1135F509968034A0A409A607047C0460040054069
S1135F60FFFF7FFF0A4B30B580245D6824040122C3
S1135F7025420AD0074D8240286802432A605A68A5
S1135F80D9609A6814439C600022101C30BDC0463E
S1135F9000400540E0FFFF1F70B5041C007BE023B8
S1135FA0984301380A2800D9A4E000F0F5FC08065B
S1135FB03932358895A3272D240000232AE04E4B3F
S1135FC080221868920502431A604C4B0020186026
S1135FD0227B1E1C4A4D910605D52169FFF7F0FA74
S1135FE023692B6004E0201C0121FFF793FC286047
S1135FF0102333607EE0434B196806E0201C002127
S1136000FFF788FC206175E02169201CFFF7D8FAAE
S113601070E00123013300E000230133013300E089
S113602000230133217B384A7F2905D915680121D2
S113603099408D4315605DE02F4980200E688005EE
S113604030432E4D08602968C80703D52C48002129
S1136050296001602D492668980046500021106887
S1136060296001219940014311602949294A022BE1
S11360700DD1294B1868234B1860284BC020187089
S113608080235B030B60116804230B4306E0244B5D
S1136090C020187080239B030B6010231360237BA4
S11360A05A0609D51F4B204A1E68002032401A6048
S11360B0134B1968FFF784FA10232B601AE0124B74
S11360C004221868002190431860201CFFF722FC6A
S11360D0114B18600023A1E7637AE12212015A43AD
S11360E0A37A3C214B43D218E37AD2180F4B1A609F
S11360F0002397E7002070BD3C80044014D0034087
S113610000D0034008D00340DCFFFF1F9CFFFF1FAB
S113611000E100E01CD00340D4FFFF1F14E400E0C2
S113612015E400E000700440FFFFF3FF98FFFF1F39
S113613008B5084B04211A680A4206D006480068CC
S1136140002802D018688843186030BF1A60FFF72F
S113615039FD08BD10ED00E0E0FFFF1F38B56C20ED
S1136160FEF7B0FD0922002310423FD020490B78EE
S1136170980604D51F4B1A780323540636D41E4BB5
S113618004201A680123024230D01A4A47241578A1
S1136190022325422AD00B789C0605D514780723C0
S11361A01C40031C022C21D00B78180705D510784D
S11361B0072318400523032818D0097801238C07E6
S11361C014D5127807210A40042A0FD10B4B1A78F0
S11361D003231A40012A08D0002A04D00823032AE2
S11361E004D0012302E0062300E00B1C181C38BD78
S11361F000E0074001E0074010ED00E002E0074046
S1136200E02208B5031C9043082853D800F0C4FBCF
S113621005080B0D1C232F3740006C2000214BE098
S11362200022274B0AE000221BE0264B20211A788B
S11362300A431A70224BC02219780A431A70224B5F
S113624004211A688A4334E01E4B20211A780A4339
S11362501A70822205E01B4B08211A780A431A702F
S11362600322174B04211A70174B1A6820E0154AB1
S113627002201178014311701F22934311E0114A47
S113628002201178014311701F229343012207E079
S11362900C4A02201178014311701F2293430322F8
S11362A013430A4A1370064B04221A70064B1968EA
S11362B00A431A606C200121FEF716FD08BDC04692
S11362C001E0074000E0074010ED00E002E0074075
S11362D0024A034B00B51A60FEE7C0460400FA0503
S11362E00CED00E010B5124A12491348891A002334
S11362F08B4203D0C45CD4540133F9E70F49104AEC
S1136300914205D10F4A10490023891A181C08E04C
S11363100E480023801A8342F4D0CC5CD454013359
S1136320F9E78B4203D0D41820700133F9E710BD8C
S113633000FEFF1F13FEFF1F4C7B0000002900001E
S11363400029000014FEFF1FBC000020326B000077
S113635008B5214B80221968D2000A431A601F4AEB
S11363601F4B21211A601F4B1A688A431A601E4B67
S11363701A6801231A401D4B00D00C221A601C4BD2
S113638008221A701B4B04221A701B4BA022197886
S11363900A431A70194B002219491A700C230A78FF
S11363A01A42FCD1174B802252021A60164A174B2C
S11363B01A60FFF797FFFCF703FE154A154B1648C2
S11363C016491A60FEF7ECFA154816490122FEF741
S11363D05BFBFEF727FCFCE7388004400301210047
S11363E080A0044054F00F4050F00F40008104405E
S11363F002D00740014006400050064000400640DD
S113640006400640448004400028000008ED00E0F7
S1136410FC050020B8000020807A0000BC000020A9
S1136420887A0000447B0000084B10B5C018802413
S113643001239C4000032243002906D0194201D0C5
S11364400260994304305B00F6E710BD4900040084
S1136450F0B5041C007985B0092800D989E200F060
S1136460A5FA0A00A5018802F60088025F028802E4
S1136470880288025C00A37958060DD45AB2002A17
S11364800CDB1025190703D52B4209D0B02508E0F1
S11364901D4007D0A02504E0802502E0C02500E0CF
S11364A090252D030222134202D003231D4302E050
S11364B05E0700D51543E679A76803960026029681
S11364C00126002F00D154E2374221D0039801283D
S11364D000D04EE223680299D04A8B506279D04BA7
S11364E09201D2B21A70CF4B802212061A60CE4BA0
S11364F080221968D2000A431A60311C2A1C0398AE
S1136500FFF792FFC94AF34311681F401940116015
S11365100298760004300290D3E7E079A568FF285A
S113652021D1C349C3480B78AB430B70227AC24BC9
S11365301A7000220123002D08D0A6681E4202D042
S113654027689D4317505B000432F4E76279BB4B24
S11365509201D2B21A70B34B80221A60A2680B78EF
S113656013430B7005E2A37918221A40083A002657
S1136570D2B20296102A02D8B149895C0291032250
S11365809F0702D45A07D20F520000280DD00128C9
S113659000D0EEE1A44B80211E68C900314319608C
S11365A0291CFFF741FFA14B09E09F4B80211E6886
S11365B0890031431960291CFFF736FFA14B1A6883
S11365C0AA431A6001220023002D00D1D1E1A06862
S11365D0104239D0E1799C4E4901C918895DFF29DF
S11365E031D003200840400003909848CF08984ECB
S11365F0381889080190891903980E780327874071
S1136600BE430E70E679904F7601F618F65D894820
S113661027680096B6003750009E072001270640E1
S1136620381CB040019FC6B23E706779834EBF01EB
S1136630FFB237707B4E802737600298039EB040CC
S11366400E7830430870954352000133BCE7814B08
S113665081491F686279394319609309012B27D056
S1136660002B02D0022B46D083E17C4B802118689A
S11366704904014319606379C0218B430CD0012B79
S113668000D076E1684B80211868C9000143196085
S113669090218900724B08E0634B80211868C9007F
S11366A00143196090216F4B890019606E4B44E0DF
S11366B06A4B80211D688904294319606379C021CC
S11366C08B430CD0012B00D053E1574B8021186829
S11366D0C9000143196090218900644B08E0524BC2
S11366E0802118688900014319609021604B89005A
S11366F01960604B21E0594B80211E68C904314365
S113670019606379C0218B430CD0012B00D030E198
S1136710454B80211868890001431960D021890004
S1136720554B08E0404B80211868890001431960EB
S1136730D021524B89001960514B3F210A40191C4A
S11367400831C020C867A17ACF060FD54D498020F3
S11367500D684004904085430D60334980200D68E6
S1136760800028430860484848490860A17A0132FB
S11367707F2903D9D1005918242002E0D1005918E7
S113678028204860A07A2189860604D549089960A2
S1136790E188490802E001399960E188D2009A1839
S11367A09160A17A3F220A401A60E2E029492A480E
S11367B00F68A37B3843A2680860012B15D0002B17
S11367C002D0022B23D0D4E00C21605E23490028A0
S11367D003DA2F4B0A6813400FE00D688020400451
S11367E028430860204D11265FE00C27E05F1B4919
S11367F0002804DA274B086803400B60B9E00D68F1
S113680080208004284308601A4D12264DE00C278E
S1136810E05F1249002841DA1F4BECE718FFFF1F25
S11368201FE400E000E100E03880044054F00F4031
S113683002C00740B4FFFF1F04C0074007E400E0A4
S1136840E87A000014F00F40327A000003C00740D9
S113685000C0074004800440000001013C80044063
S113686028A004402CA004400080034034A004402D
S113687000900440009003402C9004402890044071
S113688000A003400C80044003040000489004402E
S1136890FFFFFFFEFFFFFFFDFFFFFFFB0D688020F2
S11368A0C0042843344D0860132600212960039650
S11368B02E68370600D52960291CC0260831CE670A
S11368C02E4E0021B24205D9072902D001315208C7
S11368D0F8E72A4A2A4F89B25E00F1530291A1894E
S11368E0C90604D58020410102980843F053AA60E8
S11368F0244922689B005A50002A08D0224A617910
S11369009A580398FFF738FABB5BC82201E0BB5BD7
S113691088221343BB53BB5B1B051B0D2B6028E074
S1136920A268120607D5A37D002B22D1174B1D6840
S11369306A0052081A60A37D002B1AD1134A8021E1
S11369401668090631431160A268D70706D5930774
S1136950DB0F9B01500701D420210B43110702D503
S1136960A08A0B490880550601D580221343094AA1
S1136970D37705B0F0BDC04600A00340FFFF000080
S1136980F0FFFF1FE4FFFF1F747A00003C80044007
S113699000F0034002F0034002B471464908490084
S11369A0095C49008E4402BC7047C04603B471467A
S11369B0490840004900095A49008E4403BC704705
S11369C0002934D00123002210B488422CD301249E
S11369D02407A14204D2814202D209011B01F8E733
S11369E0E400A14204D2814202D249005B00F8E7EC
S11369F0884201D3401A1A434C08A04202D3001B18
S1136A005C0822438C08A04202D3001B9C0822434A
S1136A10CC08A04202D3001BDC082243002803D088
S1136A201B0901D00909E3E7101C10BC70470028BA
S1136A3001D00020C04307B4024802A140180290CC
S1136A4003BDC046D90000000029F0D003B5FFF70C
S1136A50B9FF0EBC4243891A1847C046002941D0E9
S1136A6010B4041C4C40A44601230022002900D584
S1136A704942002800D5404288422CD301242407EF
S1136A80A14204D2814202D209011B01F8E7E400C9
S1136A90A14204D2814202D249005B00F8E7884255
S1136AA001D3401A1A434C08A04202D3001B5C08CD
S1136AB022438C08A04202D3001B9C082243CC082A
S1136AC0A04202D3001BDC082243002803D01B0988
S1136AD001D00909E3E7101C6446002C00D54042AC
S1136AE010BC7047002806D003DB0020C0434008D8
S1136AF001E08020000607B4024802A14018029079
S1136B0003BDC046190000000029EBD003B5FFF710
S1136B10A7FF0EBC4243891A1847C0467047C046B7
S1136B2000B5031C8218934202D019700133FAE7AE
S1056B3000BDA2
S1136B344376BA6B730102030405060708090A4382
S1136B446F6E6E656374696F6E2074696D6564201D
S1136B546F75740D0A000000150078002000000011
S1136B6417005D00070000000041444D494E002019
S1136B7420755461736B6572264B494E45544953D1
S1136B840000000000000000000000000000501499
S1136B9403030000325F00004276BA6B710D0A0AE7
S1136BA448656C6C6F2C20776F726C642E2E2E20CB
S1136BB44B494E455449530D0A006E524632344CE7
S1136BC43031502B20006D61737465720D0A0073AB
S1136BD46C6176650D0A0050696E672052460D0A91
S1136BE40052544320416C61726D2066697265647D
S1136BF40D0A00444154412041434B454421210D95
S1136C040A004E6F2041434B203B2D280D0A0052AD
S1136C1478206461746120617661696C61626C6579
S1136C24202D20706970652000203A2000574F4BB6
S1136C34454E202D2000676F696E6720746F204CC9
S1136C44535320616761696E0D0A00726573746F32
S1136C5472696E672057414954206D6F64650D0A4B
S1136C64004376BA6B72436F6D6D616E64206C6918
S1136C746E6520626C6F636B65640D0A000000002E
S1136C84ED740000F07400000012000000750000B0
S1136C9405750000020000004A544147000820081A
S1136CA400000000ED740000F07400000012000005
S1136CB40075000005750000020000004C6F636B52
S1136CC4757000506F7765722D6F6E00ED7400005F
S1136CD4F074000000120000C7770000D0770000B1
S1136CE405000000E5770000EE77000005010000D0
S1136CF4067800000F7800000502000023780000E5
S1136D042B78000005030000467800004F7800004B
S1136D14050400006F7800007E780000051500006B
S1136D2499780000A7780000051600006675000035
S1136D34C4780000051100002E75000018750000C9
S1136D44000000000075000005750000020000004A
S1136D5431000000312E350032000000536F667498
S1136D64776172650074616D70657200ED74000082
S1136D74F074000000120000337500003B7500003D
S1136D84010A00004F75000056750000010100005F
S1136D942E75000018750000000000000075000046
S1136DA40575000002000000436C6F636B206C6F78
S1136DB4737300486F7374206465627567676572E2
S1136DC400000000ED740000F074000000120000E4
S1136DD4007500000575000002000000ED74000059
S1136DE4F074000000120000007500000575000036
S1136DF402000000FF710000DE78000000040000BF
S1136E04F6780000F878000000050000097200001C
S1136E1413790000000600002279000024790000A0
S1136E24000700003E7900004079000000090000DA
S1136E345F79000061790000000A000070730000AB
S1136E4470790000000E0000727300007F79000066
S1136E54000F00009A7900009C79000000100000E3
S1136E64B7790000E0740000001100002E750000E2
S1136E74187500000000000000750000057500008E
S1136E8402000000ED740000F07400000012000021
S1136E946675000072750000060200008575000026
S1136EA48F750000060A0000A1750000AA75000091
S1136EB406090000BC750000C57500000608000042
S1136EC4D9750000E4750000060C0000F675000096
S1136ED400760000060B00001A76000024760000F9
S1136EE4060D00003176000039760000011F000011
S1136EF45976000060760000012000007C760000D2
S1136F0482760000010000008F760000987600006D
S1136F14011A00002E75000018750000000000001E
S1136F2400750000057500000200000045787465D2
S1136F34726E616C00455A504F525400ED74000057
S1136F44F0740000001200002E7500001875000093
S1136F540000000000750000057500000200000038
S1136F6457444F47003330300000000036303000BF
S1136F740000003132303000000032343030000080
S1136F84003438303000000039363030000000312D
S1136F943434303000003139323030000033383486
S1136FA4303000003537363030000031313532307E
S1136FB430003233303430300057616B6575700003
S1136FC44F444400004556454E004E4F4E45003F45
S1136FD43F3F0057616B657570207265736574007B
S1136FE4ED740000F074000000120000A4760000A8
S1136FF4A7760000010F0000D4760000D7760000C5
S1137004011000000377000006770000011100005E
S1137014367700003E770000010200005C77000030
S113702464770000010B00007E770000887700007D
S1137034010400009F770000AA7700000105000006
S11370442E75000018750000000000000075000093
S113705405750000020000004E4F4E45000000007C
S11370645254530000000000584F4E00000000002A
S1137074F86D00000F0C000039740000DC79000086
S11370841402000048740000D06C0000160B0000C9
S11370945B740000E46F00000F0A00006D740000CC
S11370A4886E0000110E000080740000706D0000F2
S11370B4110500008F740000406F00000D030000F0
S11370C49E740000C86D00000D020000AB74000043
S11370D4A86C00000D020000B8740000E06D00000C
S11370E40F020000C9740000846C00000F02000049
S11370F4DD740000536F667477617265207665727F
S113710473696F6E20000A0A0D000A0D3D3D3D3D72
S11371143D3D3D3D3D3D3D3D3D3D3D3D3D3D3D0ACA
S11371240D000A0D415250207265736F6C766564CC
S11371340A0D000A0D415250207265736F6C757408
S1137144696F6E206661696C65640A0D000A0D53EB
S1137154657269616C206E756D6265723A200044D3
S11371646576696365206964656E746966696361DB
S113717474696F6E3A20004E657720616C61726D9C
S1137184207365740D0A00416C61726D20636C6533
S1137194617265640D0A004E65772074696D65201B
S11371A47365740D0A004E657720646174652073F9
S11371B465740D0A0030203D2052554E0031203DA7
S11371C420574149540032203D2053544F5000333A
S11371D4203D20564C50520034203D20564C5053F0
S11371E40035203D204C4C530036203D20564C4C59
S11371F453300037203D20564C4C53310038203D49
S113720420564C4C533300205B6163746976655D8E
S1137214004C6173742072657365742063617573C3
S113722465203D20000A0D53797374656D206D65E6
S11372346D6F7279207573653A0A0D00467265653F
S11372442068656170203D20002066726F6D200007
S11372540A0D556E7573656420737461636B203D08
S113726420000D0A546865206465766963652068A6
S11372746173206265656E206F7065726174696EF6
S11372846720666F72200042616420706F727420FC
S11372946E756D6265720D0A000D0A506F7274206A
S11372A4646972656374696F6E3A20004F55545073
S11372B455540D0A00494E5055540D0A00496E7632
S11372C4616C696420706F72740D0A00506F72747B
S11372D420697320696E7075740D0A00506F72749E
S11372E42073746174653A2000310D0A00300D0A6C
S11372F4000D0A3F3F0D0A23004D656D6F7279201E
S1137304446973706C61790D0A00202020200046C2
S1137314696C6C0D0A0057726974650D0A000A0DD4
S1137324427965204279650A0D00496E636F727271
S11373346563742064617461206C656E6774680DA0
S11373440A000D0A53657269616C20636F6E666985
S11373546775726174696F6E0D0A00426175642009
S11373643D2000696E76616C696421003700380041
S113737420426974730D0A002073746F702062696B
S1137384742873290D0A00466C6F7720636F6E743A
S1137394726F6C2000486967682077617465722095
S11373A400250D0A004C6F77207761746572200004
S11373B4656E61626C650064697361626C65000D7D
S11373C40A496E76616C6964207377697463680D25
S11373D40A00496E636F727265637420736572691F
S11373E4616C2073706565640D0A00496E636F7285
S11373F472656374207061726974790D0A00496E50
S1137404636F72726563742073746F70206269743D
S1137414730D0A00496E636F727265637420666C3F
S11374246F7720636F6E74726F6C0D0A000A0D0D12
S1137434004D41430020202020204D61696E206DC1
S1137444656E7500204C414E20636F6E66696775E6
S1137454726174696F6E0020202053657269616CD7
S113746420636F6E6669672E0020496E7075742FF1
S11374744F7574707574206D656E750020202041FD
S1137484646D696E2E206D656E7500202020537422
S11374946174732E206D656E750020202020555371
S11374A442206D656E750020202020493243206DF2
S11374B4656E750020204469736B20696E7465726F
S11374C466616365004654502F54454C4E45542020
S11374D4636F6D6D616E64730020202043414E2000
S11374E4636F6D6D616E647300757000676F2074F3
S11374F46F206D61696E206D656E750071756974B8
S1137504004C6561766520636F6D6D616E64206DFA
S11375146F646500446973706C6179206D656E7580
S11375242073706563696669632068656C700075AF
S1137534705F74696D650053686F77206F7065724E
S11375446174696E672074696D65006D656D6F7231
S1137554790053686F77206D656D6F727920757348
S1137564650073686F775F636F6E6669670053685D
S11375746F7720636F6E66696775726174696F6E85
S11375840073686F775F74696D6500446973706C28
S1137594617920646174652F74696D650073657421
S11375A45F74696D65005365742074696D65206842
S11375B4683A6D6D3A7373007365745F64617465DE
S11375C40053657420446174652064643A6D6D3AB3
S11375D4797979790073686F775F616C61726D0092
S11375E4446973706C617920616C61726D20642FDD
S11375F474007365745F616C61726D00536574200B
S1137604616C61726D20286461746529282B295B7F
S113761474696D655D0064656C5F616C61726D00B5
S113762444656C65746520616C61726D0073686F88
S1137634775F6C700053686F77206C6F7720706F7E
S1137644776572206D6F646520616E64206F707459
S1137654696F6E73007365745F6C70005B6F707434
S1137664696F6E5D20536574206C6F7720706F773B
S11376746572206D6F64650072657365740052658C
S113768473657420646576696365006C6173745F03
S11376947273740052657365742063617573650055
S11376A46D64004D656D6F727920446973706C610B
S11376B479205B616464726573735D205B3C6C3E2A
S11376C47C3C773E7C3C623E5D205B6E756D5D0068
S11376D46D6D004D656D6F7279204D6F64696679C7
S11376E4205B616464726573735D205B3C6C3E7CF7
S11376F43C773E7C3C623E5D205B76616C5D006D54
S113770466004D656D6F72792046696C6C205B610F
S11377146464726573735D205B3C6C3E7C3C773EB1
S11377247C3C623E5D205B76616C5D205B6E756DB6
S11377345D007365745F6464720053657420706FD4
S113774472742074797065205B312E2E345D205B55
S11377543C693E7C3C6F3E006765745F6464720000
S11377644765742064617461206469726563746933
S11377746F6E205B312E2E345D00726561645F7020
S11377846F7274005265616420706F727420696E44
S1137794707574205B312E2E345D007772697465C4
S11377A45F706F72740053657420706F7274206F0D
S11377B47574707574205B312E2E345D205B302F0C
S11377C4315D007365745F62617564005365742090
S11377D473657269616C2062617564207261746599
S11377E4007365745F73746F7000536574207374ED
S11377F46F7020626974732028312F312E352F3233
S113780429007365745F626974730053657420643A
S113781461746120626974732028372F38290073D6
S113782465745F7061720053657420706172697469
S11378347920284556454E2F4F44442F4E4F4E45EC
S113784429007365745F666C6F77005365742066F2
S11378546C6F7720636F6E74726F6C2028584F4E70
S11378642F5254532F4E4F4E4529007365745F684D
S11378746967685F77617465720053657420666C28
S11378846F77207374616C6C20282529205B312E5A
S11378942E39395D007365745F6C6F775F7761743B
S11378A465720053657420666C6F77207265737417
S11378B461727420282529205B312E2E39395D000C
S11378C453686F772073657269616C20636F6E66A9
S11378D4696775726174696F6E00436F6E66696778
S11378E4757265204C414E20696E746572666163DD
S11378F465003200436F6E6669677572652073654F
S11379047269616C20696E746572666163650047AF
S11379146F20746F20492F4F206D656E75003400FD
S1137924476F20746F2061646D696E69737472614A
S113793474696F6E206D656E75003500476F207431
S11379446F206F766572766965772F7374617469D5
S11379547374696373206D656E75003600476F2018
S1137964746F20555342206D656E7500476F207403
S11379746F20493243206D656E7500476F20746F24
S1137984207574464154206469736B20696E746570
S113799472666163650039004654502F54454C4E59
S11379A4455420636C69656E7420636F6D6D616EFC
S11379B464730061007065726970686572616C203B
S11379C46661696C75726500556E646572766F6C78
S11379D47461676500000000ED740000F074000039
S11379E4001200000075000005750000020000008C
S11379F456312E342E303038001F1C1F1E1F1E1FFC
S1137A041F1E1F1E1F4E6F20616C61726D20656EF8
S1137A1461626C65640011278913C509E304720269
S1137A243901D1009D004F0035001B000E00FFFFFB
S1137A34FFFFFFFFFFFFFFFFFFFFFFFFFFFFFFFF4E
S1137A44FFFFFFFFFFFFFFFFFFFFFFFFFFFF05FF38
S1137A54FFFFFFFFFFFFFFFFFFFFFFFFFFFFFFFF2E
S1137A64FFFFFFFFFFFFFFFFFFFFFFFFFFFF00001C
S1137A74B55C0000A55C0000955C000001000004F6
S1137A8400000000207B00004154000000000000BE
S1137A9404000100257B0000892B0000450002003E
S1137AA400000000297B0000F53100002500FFFFE1
S1137AB400000000347B0000595A00002500FFFF39
S1137AC4000000003B7B00008D5A00000000000011
S1137AD4000001000000000000000000000000009D
S1137AE4000000000100000000000000020000008B
S1137AF4000000000348544D004A504700474946DB
S1137B0400435353004A530042494E00545854000E
S1137B14424D500049434F003F3F3F0057646F6755
S1137B2400617070006D61696E74656E61636500F7
S1137B346B6565706572006C6F77506F7765720062
S10B7B440157616D6B6C000038
S1137B4CFF0000000100000001000000FF0401011F
S1067B5CB2070168
S9032900D3
